:10431D0000010C01010502011E030A96040132057C
:10432D00040406006407010108000009015A0E018A
:10433D00010F000112006413010114013C1501FA73
:10434D001664FA17FFFF1D0007200007240002273F
:10435D0001012F013C30030332010335FFFF36030A
:10436D00073CFFFF3DFFFF180002191E461A000211
:10437D001B00022D32C82E0001FAFAFA180000199E
:10438D00FFFF1A00001B00002D32C82E0001FAFAA3
:10439D00FA18000019FFFF1A00001B00002DFFFF87
:0643AD002EFFFFFAFAFAF0
:10004800900786E0FEA3E0FF7457BE0010D39F40E0
:100058000C90431D12001EE493F599804C900014F7
:10006800E0D394044014900786E0FEA3E0FF904399
:100078001D12001EE493F599802F900014E0D3948C
:10008800034014900786E0FEA3E0FF90433212007D
:100098001EE493F5998012900786E0FEA3E0FF9096
:1000A800434712001EE493F59990078612000E90BC
:1000B8000786E0FEA3E0FF746C6F4E7003751300B3
:1000C80022900072E0B401087402900072F0D20F1E
:1000D80090013AE090002AF090013BE090002BF06C
:1000E80090013CE090002CF0A20DB3401690013A2C
:1000F800E0700C90013BE0700690013CE0600280EB
:1001080002C20D90013AE0B4300F90013BE0B447D1
:100118000890013CE0643B60028004D20E8002C279
:100128000EE558B40102800302024B900057E0F537
:1001380066900062E0F568900063E0F569900074ED
:10014800E0F56A90007AE0900029F090007CE0F5F4
:100158006590007DE0F567900080E0F5649000818F
:10016800E0F563900090E0900041F0900091E090FD
:100178000042F0900092E0900043F0900093E090ED
:100188000044F0900094E0900045F0900095E090D5
:100198000046F0900096E0900047F0900097E090BD
:1001A8000048F0900099E0900033F090009AE090B9
:1001B8000034F090009BE0900035F090009CE090B7
:1001C8000036F0900079E0B4011790000A740FF03F
:1001D800A374FFF090000CE4F0A3F074029000798F
:1001E800F0900079E0B4035990000CE0FEA3E0FF22
:1001F80090000AE0FCA3E0FD1200037410124432E0
:100208007408124424EF900026F0EF700674FF90F3
:100218000026F07400900079F090000BE090002721
:10022800F090000AE0900028F0900026E0900789FE
:10023800F0900027E090078AF0900028E090078B64
:10024800F0803F900081E07006755801756300A248
:100258000DB3402E90013AE090002AF090013BE067
:1002680090002BF090013CE090002CF090002AE0E8
:10027800700C90002BE0700690002CE06002800269
:10028800C20DE5667003756602E56870037568025D
:100298007E817F99E5668E048F05FF1244148C39A0
:1002A8008D3AE56975F0FAA4FFAEF0E5688E048F23
:1002B80005FF1244148C3D8D3E90004FE0F5609090
:1002C800004DE0FE900069E0B5061890004CE0FE95
:1002D800900068E0B5060C90004BE0FE900059E0F5
:1002E8006E606F900069E07006900068E0600674C8
:1002F80000900059F0900069E0B402089000497439
:1003080001F08005900049E4F0900068E0B402082C
:1003180090004A7401F0800590004AE4F09000686B
:10032800E0600690004AE060028005756004800382
:10033800756005E559B55802D20F900068E0900045
:100348004CF0900069E090004DF0900059E090006A
:100358004BF0740190009EF0740090009FF07401BF
:100368009000A0F074009000A1F074009000A2F03A
:1003780074009000A3F074009000A4F07401900041
:10038800A5F074009000A6F074009000A7F0740027
:100398009000A8F074009000A9F074009000AAF0F2
:1003A80074009000ABF074019000ACF07400900001
:1003B800ADF074019000AEF074009000AFF07400DE
:1003C8009000B0F074009000B1F074009000B2F0AA
:1003D8007401900362F07400900363F0740090035A
:1003E80064F07400900365F07400900366F0740084
:1003F800900367F07400900368F074019003A2F012
:1004080074019003A3F074009003A4F074009003A7
:10041800A5F074009003A6F074009003A7F0740090
:100428009003A8F074009003E2F074019003E3F0E5
:1004380074009003E4F074009003E5F074009003F6
:10044800E6F074009003E7F074009003E8F074009D
:10045800900422F07400900423F07401900424F0B6
:100468007400900425F07400900426F07400900441
:1004780027F07400900428F07400900462F074006F
:10048800900463F07400900464F07401900465F0C3
:100498007400900466F07400900467F0740090048F
:1004A80068F022E5B554F7F5B5E5B554FDF5B5C2E4
:1004B80093C294C291C292C207C208E5B554FBF533
:1004C800B5755105E55104F55290004FE0F560907F
:1004D8000025E4F0C20CE5B554FEF5B5C28E758D65
:1004E80000758B00754C00752600752500D28E228C
:1004F800750A00750900AE09AF0A7457BE00039F5C
:1005080050030205B590431D12001EE49390004E5F
:1005180012444A0FBF00010EE0FC90431D12001E5A
:10052800ECFEE493FFEEC39F5026AE09AF0A0FBF5F
:1005380000010E90431D12001EAE09AF0AE493FCA1
:1005480090431D12001EE49390004E12444AECF0B2
:10055800AE09AF0A90431D12001EE49390004E129C
:10056800444AE0FC90431F12001EECFCE493FDECAF
:10057800D39D401990431F12001EE493FC90431D25
:1005880012001EE49390004E12444AECF0AE09AFFC
:100598000A74022FFF50010E8E098F0A780A74011F
:1005A80026F6500418E436F640030204FE22750AC3
:1005B80000750900AE09AF0A7415BE00039F500309
:1005C80002068390437412001EE49390004E124476
:1005D8004A0FBF00010EE0FC90437412001EECFEAF
:1005E800E493FFEEC39F5026AE09AF0A0FBF000188
:1005F8000E90437412001EAE09AF0AE493FC9043B8
:100608007412001EE49390004E12444AECF0AE09B6
:10061800AF0A90437412001EE49390004E12444AAD
:10062800E0FC90437612001EECFCE493FDECD39DB5
:10063800401990437612001EE493FC904374120014
:100648001EE49390004E12444AECF0AE09AF0A74CF
:100658000F6F4E7006750A15750900AE09AF0A745A
:10066800022FFF50010E8E098F0A780A740126F6B0
:10067800500418E436F640030205BC22750A0075DA
:100688000900AE09AF0A7415BE00039F50030207A4
:100698005190438912001EE49390004E12444A0F71
:1006A800BF00010EE0FC90438912001EECFEE493AB
:1006B800FFEEC39F5026AE09AF0A0FBF00010E9090
:1006C800438912001EAE09AF0AE493FC90438912D5
:1006D800001EE49390004E12444AECF0AE09AF0AB3
:1006E80090438912001EE49390004E12444AE0FCA5
:1006F80090438B12001EECFCE493FDECD39D401953
:1007080090438B12001EE493FC90438912001EE470
:100718009390004E12444AECF0AE09AF0A740F6F82
:100728004E7006750A15750900AE09AF0A74022FD6
:10073800FF50010E8E098F0A780A740126F65004BC
:1007480018E436F6400302068A22750A0075090085
:10075800AE09AF0A7415BE00039F500302081F902C
:10076800439E12001EE49390004E12444A0FBF00AD
:10077800010EE0FC90439E12001EECFEE493FFEE97
:10078800C39F5026AE09AF0A0FBF00010E90439ECB
:1007980012001EAE09AF0AE493FC90439E12001E9D
:1007A800E49390004E12444AECF0AE09AF0A90432D
:1007B8009E12001EE49390004E12444AE0FC9043BF
:1007C800A012001EECFCE493FDECD39D401990436D
:1007D800A012001EE493FC90439E12001EE4939026
:1007E800004E12444AECF0AE09AF0A740F6F4E7017
:1007F80006750A15750900AE09AF0A74022FFF5075
:10080800010E8E098F0A780A740126F6500418E43E
:1008180036F6400302075822054D22054C22054EA4
:10082800C2CF2290F800E4936406600280FE7584CB
:100838000175A70075FF80900788E4F075C91075E9
:10084800A70F75A1C775A70075D90075CEFF75A745
:100858000F75F1FE75F2FF75F33775F47875A4BA64
:1008680075A5FF75A60775AE0075AFFF75D48175C0
:10087800D5FF75D6FF75D7FFC296C295C2A0C2979D
:10088800C291C293C294E5B554DFF5B5E5B554EF0E
:10089800F5B5E5B5547FF5B5E5B554F7F5B5E5B566
:1008A80054FDF5B575A70075A20175A14775F8093E
:1008B80075BC0175BE0475BD6C75BE0775BDA075A8
:1008C800BE0875BD0175BC0075BB1875BC2075BA2E
:1008D8000875E88075D11375A70F75E10575E200F5
:1008E80075C740759700759780740A124404759708
:1008F800C0E5975420700280F8758F0275A700D262
:10090800AF75980075A90C75A70F75AB4375ADFB4E
:1009180075AC1E75A700758911758E00758C0075EC
:100928008A00D2A9D28C758D00758B00D2ABD28E7D
:1009380075CD0075CC0075CA0075CB00D2ADC2CF9D
:10094800D2CA7591047592007593CD75EF0675D965
:100958004075CF01900786E4F0A3F0751300751475
:1009680000C299D20DC2101204AB74C8F5187517DD
:1009780000122B6B75A70FE5FB90001AF0E5FA90B3
:10098800001BF0E5F990001CF075A70090F800E452
:1009980093F508122CA21231DC900789E09000260A
:1009A800F090078AE0900027F090078BE0900028ED
:1009B800F090078CE0900029F090078DE0F56690A4
:1009C800078EE0F56890078FE0F569900790E0F5ED
:1009D8006A900791E0F565900792E0F567900793B4
:1009E800E0F564900794E0F563900795E090002A9D
:1009F800F0900796E090002BF0900797E090002C7D
:100A0800F0900798E0900041F0900799E09000423C
:100A1800F090079AE0900043F090079BE090004424
:100A2800F090079CE0900045F090079DE09000460C
:100A3800F090079EE0900047F090079FE0900048F4
:100A4800F09007A0E0900033F09007A1E090003408
:100A5800F09007A2E0900035F09007A3E0900036F0
:100A6800F07400900082F090013AE0700C90013B25
:100A7800E0700690013CE060028004C20D8002D262
:100A88000D90F807E493900021F0900021E0440ACB
:100A9800900021F0900021E054FE900021F07406AF
:100AA800900012F07402900013F090F802E4939012
:100AB8000014F07403900015F07403900016F0749D
:100AC80002900017F07405900018F0900014E0B43C
:100AD80004067404900018F0900014E0B40306743F
:100AE80003900018F07405900019F090F804E4934E
:100AF80090001DF0740090001EF090F805E49390AB
:100B0800001FF090F806E493900020F074FF900026
:100B180022F0744C900125F07465900126F07478E9
:100B2800900127F07475900128F07473900129F0F2
:100B3800742090012AF0744190012BF074369001D2
:100B48002CF0743590012DF0743090012EF074451E
:100B580090012FF07420900130F07435900131F03D
:100B68007453900132F07450900133F090007AE0A1
:100B7800D394014006740090007AF07558017559B5
:100B880001740390004CF01200C91204F89000148C
:100B9800E0B404051206848011900014E0D3940494
:100BA80040051205B68003120752122B97E5B5547B
:100BB800FEF5B5900025E4F0900786E4F0A3F07503
:100BC8002400752300754800752A007529007549A9
:100BD80000753200753100754A007554007555006E
:100BE800755A0075510575520175343C7533007599
:100BF80071007570007572CD755600755700754394
:100C080000754400754500754600755B0075470022
:100C1800754200754100900006E4F0A3F0900008CA
:100C2800E4F0A3F0755E00755F0090000E74FDF0AF
:100C3800A374E8F0900023E4F07464900024F0C2F8
:100C480000D201C202D203C209756D00C20A754DF5
:100C580000756E00C2A1C2A2C287C290E5B554BF9A
:100C6800F5B5C20F7E017F00900028E01244329053
:100C78000027E02FFF50010E90000AEEF0A3EFF0DE
:100C8800900026E0700674FF900026F090000AE0BD
:100C9800FEA3E0FFEFD394FFEE940F400790000A05
:100CA800E4F0A3F07400900071F07400900079F003
:100CB8007400900082F0740090008DF07400900031
:100CC800B4F0E5677003756704743A90074EF074E2
:100CD800FD90074FF0900414E0900454F0D2B0D285
:100CE800B7D2A7D2A6D2B1D2A3C207C208A2B6B3BE
:100CF8009204A2B3B39205D29CD2EC75CF01A2980C
:100D0800B34005C298123540E5136006A299B3B303
:100D180040028005C299123AB0E51464016005E505
:100D280014B4040280D5E54DD39405400CE55AC3AC
:100D380094C85002055A754D00E572C394F0501AD4
:100D4800787012003FAE70AF71EFD394E8EE940361
:100D580040080572757100757000C28E7E047F00B0
:100D6800E54C124432E58D75F004A4FDACF0EF2D8E
:100D7800FDEE3CFCE58B75F04084FF7E00ED2FFF17
:100D8800EC3EFE8E258F26D28EA2B6300401B350DB
:100D980003020EDEA2B6300401B35003020EDEA237
:100DA800B640670554A210400575FFA0D210E5B5FE
:100DB8004401F5B5900024E4F0E554D39566404825
:100DC8007C817D99AE25AF2612423C8E238F24E587
:100DD800482FFF50010E74011244248E238F24855E
:100DE8002448755401C28E758D00758B00754C00B2
:100DF800D28E7403BE00039F50069000257401F044
:100E0800E543B40603754300D204A2B6B350030207
:100E18000EDEC20490006BE06018123BF1A200B332
:100E28004008E5B54408F5B58006E5B554F7F5B5CD
:100E38008002C20090006EE06018123D46A202B324
:100E48004008E5B54402F5B58006E5B554FDF5B5AD
:100E58008006E5B554FDF5B5A207B34004D28780F6
:100E680002C287900059E06004D2908002C290903C
:100E7800004AE0B40104D2A18002C2A1900049E076
:100E8800B40104D2A28002C2A2A20CB34008E5B504
:100E98004440F5B58006E5B554BFF5B5900018E0B7
:100EA800FE900014E0C39E4009900014E0D394081B
:100EB800400974FB900023F01204AB90001DE06021
:100EC8001590001DE0FE900017E06E600974FE901A
:100ED8000023F01204ABC2CA7E017F00E54E124423
:100EE80032E5CD2FFF50010E8E278F28D2CAE56537
:100EF800B4014890000EE0FCA3E0FDEFC39DEE9C1A
:100F08004039B20BE52A45296013A20BB34008E526
:100F1800B54404F5B58006E5B554FBF5B590000E6B
:100F2800E0FEA3E0FF900010E0FCA3E0FDEF2DFD44
:100F3800EE3CFC90000EECF0A3EDF0A2B3300501FE
:100F4800B3500302102CA2B3300501B350030210B2
:100F58002CA2B350030210250555A210400575FFB9
:100F6800A0D210E5B54401F5B5900024E4F0E555AC
:100F7800D3956850030210237CEA7D60AE27AF2822
:100F880012423C8E298F2AE56912443274FF8E047E
:100F98008F05FF1244148C298D2AE5492DFD500137
:100FA8000C74018C068D071244248E298F2A852AF9
:100FB80049A20CB340157464124432900067E08E65
:100FC800048F05FF1244148C298D2A755501900051
:100FD8000EE0FEA3E0FFAC27AD2812000390000E40
:100FE800EEF0A3EFF0E567FF124414740AFF124411
:100FF8001490007BE08C068D0712443274148E0422
:101008008F05FF124414900010ECF0A3EDF0C2CA53
:1010180075CD0075CC00754E00D2CAD205A2B3B307
:101028004002C205900025E0B40107E556C39406C6
:101038004003021BA7E56E902B38F8282873900010
:1010480059E0C39402400302119AE551D394015028
:101058000302119AE55175F040A4FFAEF090031217
:1010680012001EE0C395455018E55175F040A4FFE5
:10107800AEF090031112001EE0F52E752D0002113E
:101088009AE55175F040A4FFAEF090031012001ECF
:10109800E0C395454003021136E55175F040A4FFC1
:1010A800AEF090031112001EE55175F040A4FFAE9A
:1010B800F0E0FC90030F12001EECFEE0FFEEC39F71
:1010C800FEE5518E0475F040A4FFAEF090031012B7
:1010D800001EE0F40425458C0088F0A4FFAEF0E57E
:1010E800518F048E0575F040A4FFAEF090031212E4
:1010F800001EE55175F040A4FFAEF0E0FA90031031
:1011080012001EEAFEE0FFEEC39FFECDCCCD8E0797
:10111800124414E55175F040A4FFAEF090030F128D
:10112800001EE02DFD50010C8C2D8D2E8064E551A4
:1011380075F040A4FFAEF090030F12001EE5517544
:10114800F040A4FFAEF0E0FC90030E12001EECFE8F
:10115800E0FFEEC39F8545F0A4FFAEF0E5518F0494
:101168008E0575F040A4FFAEF090031012001EE04B
:10117800FECDCCCD8E07124414E55175F040A4FF86
:10118800AEF090030E12001EE02DFD50010C8C2DC8
:101198008D2E756E01021BA7900059E0C394024082
:1011A800030212F690004FE0D3955150030212F655
:1011B800E55175F040A4FFAEF090031812001EE050
:1011C800C395455018E55175F040A4FFAEF0900363
:1011D8001712001EE0F52C752B000212F6E551756A
:1011E800F040A4FFAEF090031612001EE0C3954530
:1011F8004003021292E55175F040A4FFAEF090034F
:101208001712001EE55175F040A4FFAEF0E0FC9007
:10121800031512001EECFEE0FFEEC39FFEE5518EA3
:101228000475F040A4FFAEF090031612001EE0F41F
:101238000425458C0088F0A4FFAEF0E5518F048E9C
:101248000575F040A4FFAEF090031812001EE5519A
:1012580075F040A4FFAEF0E0FA90031612001EEA03
:10126800FEE0FFEEC39FFECDCCCD8E07124414E501
:101278005175F040A4FFAEF090031512001EE02D4A
:10128800FD50010C8C2B8D2C8064E55175F040A429
:10129800FFAEF090031512001EE55175F040A4FF53
:1012A800AEF0E0FC90031412001EECFEE0FFEEC36B
:1012B8009F8545F0A4FFAEF0E5518F048E0575F0CB
:1012C80040A4FFAEF090031612001EE0FECDCCCD78
:1012D8008E07124414E55175F040A4FFAEF0900358
:1012E8001412001EE02DFD50010C8C2B8D2C756EF8
:1012F80002021BA7900059E0B4022AE55175F0409C
:10130800A4FFAEF090031712001EE0F52C752B0019
:10131800E55175F040A4FFAEF090030E12001EE0F8
:10132800F52E752D00900059E0B4030F900051E0A0
:10133800F52C752B00752E00752D00E551B40105AF
:10134800756E048017E551B40205756E05800DE5CC
:1013580051B40305756E068003756E03021BA7E57D
:1013680051D394034015E55175F040A4FFAEF090B9
:10137800032012001EE0C3955A4002807DAE23AFC1
:1013880024AC2DAD2EEDD39FEC9E401AE55175F09F
:1013980040A4FFAEF090031E12001EE0A829B8007A
:1013A80005D3952A500280021551E551B55237E50B
:1013B80051C395605030E55604D395514028AE236B
:1013C800AF24AC2BAD2CEFD39DEE9C4019E55175A5
:1013D800F040A4FFAEF090031F12001EE0A829B849
:1013E8000006952A400280020551C292E5516552D5
:1013F8006008C207755A00756DFA756E08021BA75A
:10140800E551B40115E55175F040A4FFAEF0900325
:101418002012001EE0C3955A40028050A209B34032
:1014280011C209755102D20AD208756DCD755A00DC
:101438008038E551C395605031AE23AF24AC2BAD55
:101448002CEFD39DEE9C400D90039FE0A829B80097
:1014580006952A40028002D209A209B3400C9003E3
:1014680060E0C39405F55A756DFAC292756E07026D
:101478001BA7E551B40215E55175F040A4FFAEF085
:1014880090032012001EE0C3955A400302152390D2
:101498000049E0701DAE23AF24AC2DAD2EEDD39FD7
:1014A800EC9E400E90039EE0A829B80005D3952A2B
:1014B80050028003755101A209B34009C209755150
:1014C80003D2088041E551C39560503AAE23AF245A
:1014D800AC2BAD2CEFD39DEE9C4014E556D3940174
:1014E800400D9003DFE0A829B80006952A40028045
:1014F80002D209A209B3400E9003A0E0C39402F5FA
:101508005A756DFAD208E5516552600D755A00E5B5
:1015180051B40105C208756DFAC292756E07021BB7
:10152800A7E551B40315E55175F040A4FFAEF0905E
:10153800032012001EE0C3955A40030215CAA209EF
:10154800B3400EC209755102D20AD208756DCD801A
:101558002DAE23AF24AC2DAD2EEDD39FEC9E400EC7
:101568009003DEE0A829B80005D3952A5002800E22
:10157800D2099003E0E0C39405F55A756DFAE55178
:10158800C395605023E556D39402401CAE23AF2484
:10159800AC2BAD2CEFD39DEE9C400D900420E0A821
:1015A80029B80006952A40028003755104E5516563
:1015B80052600DE551B40405C207756DFA755A00FD
:1015C800C292756E07021BA7E55175F040A4FFAEE5
:1015D800F090031A12001EE0B40117E55175F040AF
:1015E800A4FFAEF090032012001EE0241EC3955AFB
:1015F80040030216A0753064752F00A207B3500B84
:10160800900060E02405C3954540030216A0E5510B
:1016180075F040A4FFAEF090031D12001EE0C395C4
:10162800454064E55175F040A4FFAEF090031C12EC
:10163800001EE55175F040A4FFAEF0E0FC90031BDE
:1016480012001EECFEE0FFEEC39F8545F0A4FFAE3E
:10165800F0E5518F048E0575F040A4FFAEF09003BD
:101668001D12001EE0FECDCCCD8E07124414E551AC
:1016780075F040A4FFAEF090031B12001EE02DFD94
:1016880050010C8C2F8D30AE23AF24AC2FAD30EF32
:10169800D39DEE9C4002D207756E09021BA7E55147
:1016A80075F040A4FFAEF090031A12001EE0B401DA
:1016B80017E55175F040A4FFAEF090032012001E0C
:1016C800E0240AC3955A4003021776753064752FD3
:1016D80000A207B3500B900060E02405C395454075
:1016E80003021776E55175F040A4FFAEF090031D94
:1016F80012001EE0C395454064E55175F040A4FF13
:10170800AEF090031C12001EE55175F040A4FFAE28
:10171800F0E0FC90031B12001EECFEE0FFEEC39FFE
:101728008545F0A4FFAEF0E5518F048E0575F040B5
:10173800A4FFAEF090031D12001EE0FECDCCCD8EAE
:1017480007124414E55175F040A4FFAEF090031B56
:1017580012001EE02DFD50010C8C2F8D30AE23AFF2
:1017680024AC2FAD30EFD39DEE9C4002D207756EAE
:1017780009021BA7E55AB41603756DCDE551B402ED
:1017880005A209B3400302189BE55AC3940A507D89
:10179800900072E0B40258E54575F00284FF7E00BF
:1017A80090018012001EE0F572E54775F00A84FF8B
:1017B8007E0090024E12001EE0F55DE572255DD3B5
:1017C8009464400BE572255DC39464F572800375DB
:1017D8007200E57275F00284FF7E008F72EFC39489
:1017E800335007EF24CDF57280037572FF801CE536
:1017F8004575F00284FF7E0090018012001EE0759E
:10180800F00284FF7E00EF24CDF572807B90007299
:10181800E0B40258E54575F00284FF7E009001B2FD
:1018280012001EE0F572E54775F00A84FF7E00900D
:10183800024E12001EE0F55DE572255DD39464400A
:101848000BE572255DC39464F5728003757200E53B
:101858007275F00284FF7E008F72EFC394335007D5
:10186800EF24CDF57280037572FF801CE54575F095
:101878000284FF7E009001B212001EE075F002841F
:10188800FF7E00EF24CDF572E55AD394024004C2DE
:10189800A0C20AE551B40206A209B3B34002807B94
:1018A800900072E0B40258E54575F00284FF7E00AE
:1018B8009001B212001EE0F572E54775F00A84FF48
:1018C8007E0090024E12001EE0F55DE572255DD3A4
:1018D8009464400BE572255DC39464F572800375CA
:1018E8007200E57275F00284FF7E008F72EFC39478
:1018F800335007EF24CDF57280037572FF801CE525
:101908004575F00284FF7E009001B212001EE0755A
:10191800F00284FF7E00EF24CDF572E551B4030791
:10192800E55AC3941940030219B4900072E0B40256
:1019380058E54575F00284FF7E009001B212001E42
:10194800E0F572E54775F00A84FF7E0090024E12BA
:10195800001EE0F55DE572255DD39464400BE572E9
:10196800255DC39464F5728003757200E57275F0A5
:101978000284FF7E008F72EFC394335007EF24CDAB
:10198800F57280037572FF801CE54575F00284FFCF
:101998007E009001B212001EE075F00284FF7E0006
:1019A800EF24CDF572E55AB41602C208756E0A0224
:1019B8001BA7E551D394034006E55A640A600280E8
:1019C80003756DCDE55164026010900050E024026B
:1019D800A823B80005D3952450028002C207E55118
:1019E800B40119A209B35014E545C39405500D90EC
:1019F800035FE0A829B80006952A4002800ED209A4
:101A0800900360E0C39405F55A756DFA900059E0AB
:101A1800C39403503BE551D394014034E55175F02C
:101A280040A4FFAEF090031412001EE0A823B800F3
:101A38001FD39524401AE55175F040A4FFAEF090ED
:101A4800031F12001EE0A829B80005D3952A5002EA
:101A58008052E55164036015900049E07004155107
:101A68008009E551D3940340021551802AA209B395
:101A780050099003E0E0C3955A4002801AE545C337
:101A880094055005755101800ED2099003E0E0C31A
:101A98009405F55A756DFAE551B40108C207C208F4
:101AA800C2A0C209756E0B021BA7E551D394014071
:101AB8002FE55175F040A4FFAEF090031212001EFE
:101AC800E0C39545501AE55175F040A4FFAEF0907B
:101AD800031E12001EE0A829B80005D3952A50025B
:101AE8008033E551B40305A209B34002800ED20940
:101AF8009003E0E0C39405F55A756DCDE551640394
:101B08006013900049E0700415518009E551D394A1
:101B18000340021551E551D394034021E556C3947F
:101B280003501AE55175F040A4FFAEF090031E1261
:101B3800001EE0A829B80005D3952A50028009E5BF
:101B480051D3940340021551E551B4031FE556B42F
:101B5800011AE55175F040A4FFAEF090031E120083
:101B68001EE0A829B80005D3952A5002801AE5512D
:101B7800B40305A209B34002800ED2099003E0E045
:101B8800C39405F55A756DCD900060E0D395455026
:0F1B980009900054E0C395455002C207756E00D6
:102B38000210460211A00212FC02136702140802D6
:102B4800147A0215290215D00216A602177C02195A
:042B5800BA021AB2F1
:101BA700900059E07003021DFCA2A5B34008A2A44F
:101BB700B34003021DE5AE35AF367441D39F749C25
:101BC7009E4005783512003FAE35AF36EFB4880634
:101BD700EEB413028003021DA7A2A55003021CD670
:101BE700900059E0B4010B90004FE0D3956040029C
:101BF7000560900059E0B4027590004FE0D395510D
:101C07004019E55175F040A4FFAEF090031412009F
:101C17001EE0A823B8000695244002804BE551B486
:101C2700010ED209900360E0C39405F55A756DFA69
:101C3700E551B40207E556D3940150028010D2094A
:101C47009003A0E0C39405F55A756DFAD208E551E3
:101C5700D394024007E556D394025002800A0551F7
:101C6700C207755A00756DFA90004FE0F560900055
:101C770059E0B4035A90004FE0D39551404BE551DA
:101C8700B4010ED209900360E0C39405F55A756D4F
:101C9700FAE551B40207E556D3940150028013D2F6
:101CA700099003A0E0C39405F55A756DFAD208753B
:101CB7005A00E551D394024007E556D394025002E7
:101CC70080070551C207756DFA90004FE0F560A2D5
:101CD700A45003021DA7900059E0B40150E551D369
:101CE70094014046E55175F040A4FFAEF090031E05
:101CF70012001EE0A829B8002CD3952A4027E551E9
:101D0700B40313D2099003E0E0C39405F55A756D47
:101D1700FA756002800D1551855160756DFA755A17
:101D270000C20880038551608003756001900059E7
:101D3700E0D39401405EE551D394014034E55175F9
:101D4700F040A4FFAEF090031112001EE0A823B8E4
:101D5700001FD39524401AE55175F040A4FFAEF05B
:101D670090031E12001EE0A829B80005D3952A503B
:101D7700028021E551B40310D2099003E0E0C39437
:101D870005F55A756DFA800C1551756DFA755A007F
:101D9700C207C208E556B40704055E8003755E00F6
:101DA700E563B4010EAE35AF36EF64407005EE64FF
:101DB7009C6002800EA2A54003755801A2A44003AF
:101DC700755802E563B4020EAE35AF36EF64407066
:101DD70005EE649C6002800690004FE0F560A2A5C6
:101DE700B3B35006A2A4B3B340028006753600759C
:101DF7003500021EFDA2A5B34008A2A4B34003020A
:101E07001EE9AE35AF367441D39F749C9E4005786A
:101E17003512003FAE35AF36EFB48806EEB4130285
:101E27008003021EE9A2A5406F900068E0605A9007
:101E3700004AE0B4010790004AE4F0800690004AA7
:101E47007401F090004AE0700575600480037560C6
:101E57000590004AE0B40104D2A18002C2A1E55175
:101E6700B4051AE55175F040A4FFAEF090031E12B9
:101E7700001EE0A829B80005D3952A5002800875EE
:101E87005104C207755A008003756005E556B4070B
:101E970004055E8003755E00A2A44046900069E0D9
:101EA7006034900049E0B40107900049E4F08006EF
:101EB7009000497401F0900049E0B40117D2A2E5FF
:101EC70051B4010ED209900360E0C39405F55A7529
:101ED7006DFA8002C2A2E556B40704055E80037559
:101EE7005E00A2A5B3B35006A2A4B3B34002800616
:101EF700753600753500E55865596006900082E033
:101F07006003022085C29C751400751300C2CAE5E0
:101F170058902B5CF828287380121231DC800D1240
:0C1F270032B5800812338E80031234673C
:0F2B5C00021F1F021F21021F26021F2B021F3004
:101F3300900029E090007AF0E566900057F0E5689C
:101F4300900062F0E569900063F0E56A900074F038
:101F5300E56590007CF0E56790007DF0E564900016
:101F630080F0E563900081F090002AE090013AF060
:101F730090002BE090013BF090002CE090013CF0AE
:101F8300900041E0900090F0900042E0900091F0CA
:101F9300900043E0900092F0900044E0900093F0B2
:101FA300900045E0900094F0900046E0900095F09A
:101FB300900047E0900096F0900048E0900097F082
:101FC300900033E0900099F0900034E090009AF094
:101FD300900035E090009BF0900036E090009CF07C
:101FE3007400900082F0744C900125F074659001A8
:101FF30026F07478900127F07475900128F07473BB
:10200300900129F0742090012AF0744190012BF083
:10201300743690012CF0743590012DF074309001DA
:102023002EF0744590012FF07420900130F0743538
:10203300900131F07453900132F07450900133F0F9
:10204300900414E0900454F0743A90074EF074FD39
:1020530090074FF01200C9900004E4F0A3F0900041
:10206300067475F0A37430F09000087475F0A374CF
:1020730030F0855859D2CA754C00D29C741B90001D
:1020830023F0E556C394065005E551B552030221EA
:102093001BC207E55175F040A4FFAEF09003221276
:1020A300001EE030E003D38001C39296E55175F042
:1020B30040A4FFAEF090032312001EE030E003D3F0
:1020C3008001C39295E55175F040A4FFAEF09003F3
:1020D3002412001EE030E003D38001C392A0E55137
:1020E30075F040A4FFAEF090032512001EE030E02F
:1020F30003D38001C39297A20AB34002D2A08551B1
:1021030052AE29AF2A7405BE00039F5007E545D39D
:10211300940550028002D292E556D39405500302EF
:102123002268C207E551D3940150030221BDE55152
:1021330075F040A4FFAEF090031E12001EE0A82924
:10214300B80007D3952A40021551E55165526067DF
:10215300E55175F040A4FFAEF090032212001EE09B
:1021630030E003D38001C39296E55175F040A4FF9C
:10217300AEF090032312001EE030E003D38001C3CE
:102183009295E55175F040A4FFAEF0900324120040
:102193001EE030E003D38001C392A0E55175F04007
:1021A300A4FFAEF090032512001EE030E003D380BD
:1021B30001C39297855152022268E556B4063490C2
:1021C30000ACE030E003D38001C392969000ADE011
:1021D30030E003D38001C392959000AEE030E0037A
:1021E300D38001C392A09000AFE030E003D380011D
:1021F300C39297E556B407349000A5E030E003D3CB
:102203008001C392969000A6E030E003D38001C31F
:1022130092959000A7E030E003D38001C392A09091
:1022230000A8E030E003D38001C39297E556B408D9
:102233003490009EE030E003D38001C39296900077
:102243009FE030E003D38001C392959000A0E0307B
:10225300E003D38001C392A09000A1E030E003D358
:102263008001C39297E54575F00284FF7E009001DB
:102273004E12001EE075F00284FF7E00EF24CDF5C0
:102283005CE595C3955C4004C2938002D293A20897
:10229300B34002800FA207B34007E556D39405402D
:1022A300037572CDE595C395724004C2948002D242
:1022B30094E595C3956D4004C2918002D291E543A4
:1022C300C3940640030228C4A2EDB350030228C4FA
:1022D300C2EDE54360030224267E017F00E5BE12C2
:1022E3004432E5BD2FFF50010E900000EEF0A3EF46
:1022F300F0900029E0B401177E0F7FFF900000E00B
:10230300FCA3E0FD120003900000EEF0A3EFF090B9
:102313000079E0B4025B900000E0FEA3E0FF9000D0
:102323000AE0FCA3E0FDEDD39FEC9E400F9000007C
:10233300E0F8A3E090000AC8F0A3C8F0900000E022
:10234300FEA3E0FF90000CE0FCA3E0FDEFD39DEEC5
:102353009C400F900000E0F8A3E090000CC8F0A3AD
:10236300C8F0900000E0FEA3E0FF74041244248F41
:1023730044900079E07060900000E0FEA3E0FF90DD
:10238300000AE0FCA3E0FDEFD39DEE9C400D12009C
:1023930003900000EEF0A3EFF08007900000E4F05C
:1023A300A3F0900000E0FEA3E0FF7410124432900B
:1023B3000026E08E048F05FF124414900000ECF019
:1023C300A3EDF07400D39D74019C4008900001E0DC
:1023D300F54480037544FFE54475F00AA4FFAEF0AD
:1023E30074198E048F05FF1244148D45ED2532FFB9
:1023F300AE3150010E74011244248F458545327568
:102403003100EFD394624003754562900072E0643B
:10241300016006900066E060028005754301800359
:1024230075BB17E543B4010280030225167E017FC5
:1024330000E5BE124432E5BD2FFF50010E900000AF
:10244300EEF0A3EFF0900072E0B4017EE534453383
:102453006025AC33AD341DBDFF011C8F028E038C90
:10246300068D07903F6812002EE493FE740193FFDC
:10247300EFC39AEE9B40028005783312445CAE337F
:10248300AF3474B3BE0025D39F4021900000E0FC1D
:10249300A3E0FD0FBF00010E903F6812002EE493EE
:1024A300FE740193FFEDC39FEC9E400280057833D9
:1024B30012003FAE33AF34E56A12443274648E04C3
:1024C3008F05FF1244148D478033900066E0602D22
:1024D300900000E0FEA3E0FFEFD39400EE940840E9
:1024E3000F900066E0B40104C20C8002D20C800D90
:1024F300900066E0B40104D20C8002C20C9000721A
:10250300E064026006900066E0600575BB16800318
:10251300754302E543B4020280030226047E017F71
:1025230000E5BE124432E5BD2FFF50010E900000BE
:10253300EEF0A3EFF0900072E0B4027EE534453391
:102543006025AC33AD341DBDFF011C8F028E038C9F
:10255300068D079040D212002EE493FE740193FF80
:10256300EFC39AEE9B40028005783312445CAE338E
:10257300AF3474B3BE0025D39F4021900000E0FC2C
:10258300A3E0FD0FBF00010E9040D212002EE49392
:10259300FE740193FFEDC39FEC9E400280057833E8
:1025A30012003FAE33AF34E56A12443274648E04D2
:1025B3008F05FF1244148D478033900066E0602D31
:1025C300900000E0FEA3E0FFEFD39400EE940840F8
:1025D3000F900066E0B40104C20C8002D20C800D9F
:1025E300900066E0B40104D20C8002C20C90007229
:1025F300E07003754700900066E07002C20C75BB83
:102603001FE543B403457E017F00E5BE124432E576
:10261300BD2FFF50010E900000EEF0A3EFF0740900
:1026230012443274E68E048F05FF1244148C418DDC
:1026330042E54A2DFD50010C74018C068D071244AE
:10264300248E418F4285424A75BB19E543B4040287
:1026530080030227AC7E017F00E5BE124432E5BD54
:102663002FFF50010E900000EEF0A3EFF074041260
:1026730044248F4BE564B401028003022739756B50
:1026830000756B00E56BD394074003022726E56BC7
:1026930090004112444AE0D3954B501AE56B9000E9
:1026A3004112444AE0F404254BFEE56B90003712D7
:1026B300444AEEF08017E56B90004112444AE0C3B0
:1026C300954BFEE56B90003712444AEEF0E56BC381
:1026D30094044009900084E0C3956B503BE56B6024
:1026E30029E56B90003712444AFEE0FFEE90003F6D
:1026F300E0D39F4013E56B90003712444AE090000B
:102703003FF0E56B900040F0800E900037E09000C2
:102713003FF07400900040F0786B740126F640039C
:10272300022687900040E0F4042408F556E556D3CA
:1027330094054002C292E564D39401402FE54BD344
:10274300946E4004D2118002C211755605E564B43B
:102753000205A211B340028003755607E564B40372
:1027630006A211B3B340028003755607E5576556B9
:102773006008E55104F552855657E556B40708E558
:10278300B54480F5B58006E5B5547FF5B5E55664E7
:10279300066005E556B40808E5B54410F5B58006AE
:1027A300E5B554EFF5B575BB13E543B405028003F6
:1027B3000228C07E017F00E5BE124432E5BD2FFF33
:1027C30050010E900000EEF0A3EFF07404124424C5
:1027D3008F46E563B4020280030228BD756B007562
:1027E3006B00E56BD394034003022874E56B900000
:1027F3003312444AE0D39546501AE56B90003312E6
:10280300444AE0F4042546FEE56B90002D12444A49
:10281300EEF08017E56B90003312444AE0C395460F
:10282300FEE56B90002D12444AEEF0E56B6029E55E
:102833006B90002D12444AFEE0FFEE900031E0D38E
:102843009F4013E56B90002D12444AE0900031F055
:10285300E56B900032F0800E90002DE0900031F097
:102863007400900032F0786B740126F6400302275F
:10287300E5900082E07043E52A45296036E558C3B8
:102883009403500A900032E004C39403400280078B
:10289300900032E004F558E558D39402400A9000C2
:1028A30032E004D3940250028007900032E004F532
:1028B300588007900032E004F55875BB180543D2E1
:1028C300ECE55ED3940450030229F075CF01C29363
:1028D300AE35AF367488D39F74139E4005A2A5B35B
:1028E3004014AE35AF367488D39F74139E4005A24F
:1028F300A4B340028058783512003FAE35AF36EFAF
:10290300B4884BEEB41347A2A5B3500990004FE02F
:10291300D395515002800C0551E551B40203755112
:10292300038011A2A5B3500890004FE065516002E7
:102933008002D207A2A4B35007E551D394015002F9
:10294300800C1551E551B40203755101C207A2A5CC
:10295300B3B35006A2A4B3B3400280067536007524
:102963003500E55165526069E55175F040A4FFAE4D
:10297300F090032212001EE030E003D38001C392E3
:1029830096E55175F040A4FFAEF090032312001EAC
:10299300E030E003D38001C39295E55175F040A484
:1029A300FFAEF090032412001EE030E003D3800159
:1029B300C392A0E55175F040A4FFAEF09003251239
:1029C300001EE030E003D38001C39297C294855187
:1029D30052A20740057572CD80037572FFE595C35A
:1029E30095724004C2948002D2940228CEA210B3FE
:1029F300500DAE25AF2674E8C39F74039E4002803A
:102A03000575FFA0D210AE25AF26EFD39420EE9428
:102A13004E5003022B0C1204ABC28E758D00758BC6
:102A230000754C00D28EC207757100757000757207
:102A3300CD755105752400752300755400755A0032
:102A4300C287900059E06004D2908002C290900047
:102A53004AE0B40104D2A18002C2A1900049E0B4CB
:102A63000104D2A28002C2A2A20CB34008E5B5447D
:102A730040F5B58006E5B554BFF5B590006BE06051
:102A830018123BF1A200B34008E5B54408F5B58040
:102A930006E5B554F7F5B58002C20090006EE0601C
:102AA30018123D46A202B34008E5B54402F5B580CD
:102AB30006E5B554FDF5B58006E5B554FDF5B590CD
:102AC300000E74FDF0A374E8F0E543B40603754308
:102AD30000900025E4F0752600752500758D0075BE
:102AE3008B00754C00900024E0C3940350089000C1
:102AF30024E004F080067403900024F0900024E0A6
:102B0300B40306E5B554FEF5B5AE27AF28EFD3946D
:102B130010EE9427401CC2CA75CD0075CC007528F1
:102B230000752700D2CA754E00752A0075290075F5
:052B33005500020D0336
:103EF80000000100013201640196019602000212DD
:103F080002240200020003000340038003C00400EF
:103F18000440048004C005000600060006000600F0
:103F2800060006000600060000FF01310163019546
:103F380001FF01FF0211022302FF02FF02FF033FFC
:103F4800037F03BF03FF043F047F04BF04FF05FF93
:103F580006FF06FF06FF06FF06FF06FF06FF06FF31
:103F68000FAA0FA50F9F0F9A0F940F8D0F870F8021
:103F78000F780F710F680F600F570F4E0F450F3BEB
:103F88000F300F250F1A0F0E0F020EF50EE80EDB7D
:103F98000ECC0EBE0EAE0E9F0E8E0E7D0E6C0E5A01
:103FA8000E470E340E200E0C0DF70DE20DCB0DB59D
:103FB8000D9D0D850D6D0D540D3A0D200D050CE967
:103FC8000CCE0CB10C940C760C580C3A0C1B0BFB59
:103FD8000BDB0BBB0B9A0B790B570B350B130AF149
:103FE8000ACE0AAB0A870A640A400A1C09F809D4EF
:103FF80009B0098C09670943091F08FB08D608B2EC
:10400800088E086A0846082307FF07DC07B90796E1
:1040180007730751072F070D06EC06CA06AA06897B
:1040280006690649062A060A05EC05CD05B005927B
:1040380005750558053C0520050504EA04CF04B5B7
:10404800049C04820469045104390422040B03F417
:1040580003DE03C803B2039D038903750361034D9F
:10406800033B03280316030402F202E102D102C053
:1040780002B002A00291028202730265025702494D
:10408800023C022F02220216020901FD01F201E69A
:1040980001DB01D001C601BB01B101A7019D01945B
:1040A800018B01820179017001680160015801509A
:1040B8000148014101390132012B0125011E011876
:1040C8000111010B010500FF00FA0FA60FA00F99BF
:1040D8000F920F8B0F840F7C0F740F6B0F620F58AA
:1040E8000F4E0F430F380F2C0F1F0F120F050EF72F
:1040F8000EE80ED80EC80EB70EA50E930E800E6CE5
:104108000E580E420E2C0E150DFD0DE40DCB0DB103
:104118000D950D790D5D0D3F0D200D010CE10CC0C5
:104128000C9E0C7C0C590C350C100BEA0BC40B9E26
:104138000B760B4F0B260AFD0AD40AAA0A800A55E9
:104148000A2A09FF09D409A8097C0950092508F990
:1041580008CD08A10875084A081E07F307C8079D77
:1041680007730749072006F706CE06A6067E0657F8
:104178000630060A05E405BF059B05770554053298
:10418800051004EF04CE04AE048F04710453043503
:10419800041903FD03E203C703AD0394037B036320
:1041A800034B0334031E030802F302DE02CA02B6FD
:1041B80002A30291027F026D025C024C023C022CB7
:1041C800021D020E020001F201E401D701CA01BE7C
:1041D80001B101A6019A018F0185017A017001667A
:1041E800015D0153014A01410139013101290121D0
:1041F80001190112010B010400FD00F700F000EAAB
:1042080000E400DE00D900D300CE00C900C400BF1E
:1042180000BA00B500B100AD00A800A400A0009C41
:10422800009900950091008E008A00870084008123
:04423800007E007B89
:102B6B00751A00751900AE19AF1AAC17AD18EDC375
:102B7B009FEC9E401674FF12440475CF01781A74B3
:102B8B000126F6500418E436F650DB22900786E453
:102B9B00F0A3F0751000750F00751300751400C2CB
:102BAB0012D21322C2AF75D900758F0375B7A575F5
:102BBB00B7F190F800E4F0758F0175B7A575B7F113
:102BCB00E50890F800F075B7A575B7F190F801E43A
:102BDB00F075B7A575B7F190079DE090F802F07509
:102BEB00B7A575B7F19007A1E090F803F075B7A5FD
:102BFB0075B7F190079EE090F804F075B7A575B71F
:102C0B00F190079FE090F805F075B7A575B7F190B7
:102C1B0007A0E090F806F075B7A575B7F19007A27D
:102C2B00E090F807F0758F0075D940D2AF2290076E
:102C3B0088E0B4AB61C2AF75D90075B62275F522C9
:102C4B00758F0375B7A575B7F1740090F600F07525
:102C5B008F01750A00750900AE09AF0A7413BE0027
:102C6B00279F402475B7A575B7F190078912001EF1
:102C7B00E0FC90F60012001EECF0780A740126F6C8
:102C8B00500418E436F650D0758F0075F51175B6F3
:102C9B002075D940D2AF22C2AF75D90075F5227518
:102CAB000A00750900AE09AF0A7413BE00229F40DB
:102CBB001F90F60012001EE493FC90078912001E71
:102CCB00ECF0780A740126F6500418E436F650D569
:102CDB0075F51175D940D2AF22900788E0B4AA02DE
:102CEB008003022E21C2AF75D90075B62275F5226D
:102CFB00758F0375B7A575B7F1740090EE00F0757D
:102D0B00B7A575B7F1740090F000F075B7A575B75E
:102D1B00F1740090F200F075B7A575B7F1740090DF
:102D2B00F400F0758F01750A00750900AE09AF0A42
:102D3B0074FFC39F74019E402475B7A575B7F190BE
:102D4B00004E12001EE0FC90EE0012001EECF0781C
:102D5B000A740126F6500418E436F650CF750A00B3
:102D6B00750900AE09AF0A74FFC39F74019E40241E
:102D7B0075B7A575B7F190024E12001EE0FC90F0EE
:102D8B000012001EECF0780A740126F6500418E4C9
:102D9B0036F650CF750A00750900AE09AF0A74FFFD
:102DAB00C39F74019E402475B7A575B7F190044E6F
:102DBB0012001EE0FC90F20012001EECF0780A7478
:102DCB000126F6500418E436F650CF750A00750943
:102DDB0000AE09AF0A74FFC39F74019E402475B700
:102DEB00A575B7F190064E12001EE0FC90F4001290
:102DFB00001EECF0780A740126F6500418E436F63F
:102E0B0050CF758F0075F51175B62075D940D2AFBF
:102E1B00743A90074EF022900788E0B4AA02800320
:102E2B00022F5FC2AF75D90075B62275F522758F6B
:102E3B000375B7A575B7F1740090E600F075B7A5EB
:102E4B0075B7F1740090E800F075B7A575B7F1741C
:102E5B000090EA00F075B7A575B7F1740090EC001F
:102E6B00F0758F01750A00750900AE09AF0A74FF82
:102E7B00C39F74019E402475B7A575B7F190004EA2
:102E8B0012001EE0FC90E60012001EECF0780A74B3
:102E9B000126F6500418E436F650CF750A00750972
:102EAB0000AE09AF0A74FFC39F74019E402475B72F
:102EBB00A575B7F190024E12001EE0FC90E80012CF
:102ECB00001EECF0780A740126F6500418E436F66E
:102EDB0050CF750A00750900AE09AF0A74FFC39F86
:102EEB0074019E402475B7A575B7F190044E12007E
:102EFB001EE0FC90EA0012001EECF0780A7401262A
:102F0B00F6500418E436F650CF750A00750900AE7A
:102F1B0009AF0A74FFC39F74019E402475B7A57552
:102F2B00B7F190064E12001EE0FC90EC0012001E52
:102F3B00ECF0780A740126F6500418E436F650CFFC
:102F4B00758F0075F51175B62075D940D2AF743AEF
:102F5B0090074EF022900788E0B4AA02800302305B
:102F6B009DC2AF75D90075B62275F522758F0375A5
:102F7B00B7A575B7F1740090DE00F075B7A575B7FE
:102F8B00F1740090E000F075B7A575B7F17400907F
:102F9B00E200F075B7A575B7F1740090E400F07519
:102FAB008F01750A00750900AE09AF0A74FFC39F44
:102FBB0074019E402475B7A575B7F190004E1200B1
:102FCB001EE0FC90DE0012001EECF0780A74012665
:102FDB00F6500418E436F650CF750A00750900AEAA
:102FEB0009AF0A74FFC39F74019E402475B7A57582
:102FFB00B7F190024E12001EE0FC90E00012001E92
:10300B00ECF0780A740126F6500418E436F650CF2B
:10301B00750A00750900AE09AF0A74FFC39F7401EE
:10302B009E402475B7A575B7F190044E12001EE0B3
:10303B00FC90E20012001EECF0780A740126F650A8
:10304B000418E436F650CF750A00750900AE09AFC7
:10305B000A74FFC39F74019E402475B7A575B7F121
:10306B0090064E12001EE0FC90E40012001EECF0E5
:10307B00780A740126F6500418E436F650CF758F93
:10308B000075F51175B62075D940D2AF743A90071B
:10309B004EF022900788E0B4AA0280030231DBC213
:1030AB00AF75D90075B62275F522758F0375B7A567
:1030BB0075B7F1740090D600F075B7A575B7F174BC
:1030CB000090D800F075B7A575B7F1740090DA00D1
:1030DB00F075B7A575B7F1740090DC00F0758F0132
:1030EB00750A00750900AE09AF0A74FFC39F74011E
:1030FB009E402475B7A575B7F190004E12001EE0E7
:10310B00FC90D60012001EECF0780A740126F650E3
:10311B000418E436F650CF750A00750900AE09AFF6
:10312B000A74FFC39F74019E402475B7A575B7F150
:10313B0090024E12001EE0FC90D80012001EECF024
:10314B00780A740126F6500418E436F650CF750A47
:10315B0000750900AE09AF0A74FFC39F74019E404E
:10316B002475B7A575B7F190044E12001EE0FC90C4
:10317B00DA0012001EECF0780A740126F6500418DF
:10318B00E436F650CF750A00750900AE09AF0A7424
:10319B00FFC39F74019E402475B7A575B7F19006C8
:1031AB004E12001EE0FC90DC0012001EECF0780AC0
:1031BB00740126F6500418E436F650CF758F00755F
:1031CB00F51175B62075D940D2AF743A90074EF011
:1031DB0022C2AF75D90075F522750A00750900AECC
:1031EB0009AF0A74FFC39F74019E401F90EE00123B
:1031FB00001EE493FC90004E12001EECF0780A7453
:10320B000126F6500418E436F650D4750A007509F9
:10321B0000AE09AF0A74FFC39F74019E401F90F06C
:10322B000012001EE493FC90024E12001EECF0788C
:10323B000A740126F6500418E436F650D4750A00C9
:10324B00750900AE09AF0A74FFC39F74019E401F3E
:10325B0090F20012001EE493FC90044E12001EEC40
:10326B00F0780A740126F6500418E436F650D4753B
:10327B000A00750900AE09AF0A74FFC39F74019E63
:10328B00401F90F40012001EE493FC90064E1200B7
:10329B001EECF0780A740126F6500418E436F6504A
:1032AB00D475F51175D940D2AF22C2AF75D900755F
:1032BB00F522750A00750900AE09AF0A74FFC39FAA
:1032CB0074019E401F90E60012001EE493FC9000D8
:1032DB004E12001EECF0780A740126F6500418E426
:1032EB0036F650D4750A00750900AE09AF0A74FFA3
:1032FB00C39F74019E401F90E80012001EE493FCD4
:10330B0090024E12001EECF0780A740126F650045F
:10331B0018E436F650D4750A00750900AE09AF0AE9
:10332B0074FFC39F74019E401F90EA0012001EE4BD
:10333B0093FC90044E12001EECF0780A740126F6F2
:10334B00500418E436F650D4750A00750900AE091E
:10335B00AF0A74FFC39F74019E401F90EC001200D4
:10336B001EE493FC90064E12001EECF0780A7401DA
:10337B0026F6500418E436F650D475F51175D9407D
:10338B00D2AF22C2AF75D90075F522750A00750947
:10339B0000AE09AF0A74FFC39F74019E401F90DEFD
:1033AB000012001EE493FC90004E12001EECF0780D
:1033BB000A740126F6500418E436F650D4750A0048
:1033CB00750900AE09AF0A74FFC39F74019E401FBD
:1033DB0090E00012001EE493FC90024E12001EECD3
:1033EB00F0780A740126F6500418E436F650D475BA
:1033FB000A00750900AE09AF0A74FFC39F74019EE2
:10340B00401F90E20012001EE493FC90044E120049
:10341B001EECF0780A740126F6500418E436F650C8
:10342B00D4750A00750900AE09AF0A74FFC39F7407
:10343B00019E401F90E40012001EE493FC90064E88
:10344B0012001EECF0780A740126F6500418E436CC
:10345B00F650D475F51175D940D2AF22C2AF75D9DC
:10346B000075F522750A00750900AE09AF0A74FFE5
:10347B00C39F74019E401F90D60012001EE493FC64
:10348B0090004E12001EECF0780A740126F65004E0
:10349B0018E436F650D4750A00750900AE09AF0A68
:1034AB0074FFC39F74019E401F90D80012001EE44E
:1034BB0093FC90024E12001EECF0780A740126F673
:1034CB00500418E436F650D4750A00750900AE099D
:1034DB00AF0A74FFC39F74019E401F90DA00120065
:1034EB001EE493FC90044E12001EECF0780A74015B
:1034FB0026F6500418E436F650D4750A0075090008
:10350B00AE09AF0A74FFC39F74019E401F90DC008D
:10351B0012001EE493FC90064E12001EECF0780A8B
:10352B00740126F6500418E436F650D475F511756F
:10353B00D940D2AF22E51464046006E59964FF60BC
:10354B00028031A2124004D2128027E51460087465
:10355B00E62514900023F0E513600874F025139012
:10356B000023F0E514B4010280FE751400751300FE
:10357B00C2128002C212E514903E9BF82828737584
:10358B001400E599B4FF03751301E599B4FE0375B7
:10359B001302E599B4FD03751303E599B4FC0375A8
:1035AB001304E599B4FA03751305E599B4FB067595
:1035BB0014011204ABE599B4F9067514041204ABAB
:1035CB00E599D394E54007E599C394F04002801642
:1035DB008599157514027E017F00E515C394E612DB
:1035EB0044328E0D8F0E900786E4F0A3F0E599D34D
:1035FB0094C44007E599C394E64002802885991549
:10360B0075140374E5C39515F50E750D00AE0DAF6E
:10361B000E903EF812002EE493F8740193900786F7
:10362B00C8F0A3C8F0D299023AAF900786E0FEA388
:10363B00E0FFEFC39400EE94054009EFD394FFEE47
:10364B0094064013900786E0FEA3E0FF90004E1215
:10365B00001EE599F0800385996C90078612000E89
:10366B00900786E0FEA3E0FFEFB40106EEB407027D
:10367B0080030238BF90074EE0B43C02800302384F
:10368B00BFA20DB35005A20EB340030237B2C29CCA
:10369B0090007AE090078CF0900057E090078DF047
:1036AB00900062E090078EF0900063E090078FF03F
:1036BB00900074E0900790F090007CE0900791F000
:1036CB0090007DE0900792F0900080E0900793F0DF
:1036DB00900081E0900794F090013AE0900795F00C
:1036EB0090013BE0900796F090013CE0900797F03B
:1036FB00900090E0900798F0900091E0900799F07F
:10370B00900092E090079AF0900093E090079BF066
:10371B00900094E090079CF0900095E090079DF04E
:10372B00900096E090079EF0900097E090079FF036
:10373B00900099E09007A0F090009AE09007A1F01C
:10374B0090009BE09007A2F090009CE09007A3F004
:10375B007400900082F01200C974AB900788F012CD
:0A376B002C3974AA900788F0E55885
:063E9B0002358A023635F3
:10377500903EBCF82828738012122CE4800D122E7E
:0B378500228008122F60800312309E8B
:0F3EBC0002377C02377E02378302378802378D48
:10379000900788E4F090013AE0700C90013BE070F3
:1037A0000690013CE060028004C20D8002D20D024E
:1037B00038B4C29C900078E0900789F090005EE0F9
:1037C00090078AF090005FE090078BF090007AE01D
:1037D00090078CF0900057E090078DF0900062E029
:1037E00090078EF0900063E090078FF0900074E0F7
:1037F000900790F090007CE0900791F090007DE0C1
:10380000900792F0900080E0900793F0900081E0A4
:10381000900794F090013AE0900795F090013BE01A
:10382000900796F090013CE0900797F0900090E0B0
:10383000900798F0900091E0900799F0900092E046
:1038400090079AF0900093E090079BF0900094E02E
:1038500090079CF0900095E090079DF0900096E016
:1038600090079EF0900097E090079FF0900099E0FD
:103870009007A0F090009AE09007A1F090009BE0E4
:103880009007A2F090009CE09007A3F074009000D5
:1038900082F074AB900788F0122C3974AA900788D4
:1038A000F0122CE4122E22122F6012309ED29C7540
:1038B00099FB80FED29C7514007513007599FB026C
:1038C0003AAF900786E0FEA3E0FFEF4E70068599C1
:1038D00010750F00900786E0FEA3E0FF74016F4EA5
:1038E000701BAC0FAD10AA0DAB0EED2BFBEC3AFA32
:1038F0008A068B0790004E12001EE599F09007860D
:1039000012000E900786E0FEA3E0FF74026F4E7077
:103910000C1200C9851599751400751300023AAF91
:10392000900786E0FEA3E0FF90004E12001EE5998E
:10393000F090078612000E900786E0FEA3E0FFAC31
:103940000DAD0E8F028E038C068D07903F30120056
:103950002EE493F9740193FEEAD39EEB9940098516
:103960001599751400751300023AAF900786E0FEB2
:10397000A3E0FF90004E12001EE599F0900786121A
:10398000000E900786E0FEA3E0FFEFB40006EEB461
:1039900001028003023AAF90001CE0D394C7400BB1
:1039A00090001CE0C394C8F516801A90001CE0D368
:1039B0009463400B90001CE0C39464F5168006905D
:1039C000001CE0F516E51675F002A4FFAEF08F6B53
:1039D000EF90004E12444AEFFCE0FDEC90005112D3
:1039E000444AEDFCE0FDEC2DB516028003023AA13D
:1039F0000FEF90004E12444AE56BFFE0FCEF9000A1
:103A00005212444AECFFE0FCEFC39CB5160280035F
:103A1000023AA1E56B90005012444AE56BFFE0FCCE
:103A2000EF90005312444AECFFE0FCEF2CB5167106
:103A3000E56B90005412444AE0C3951690079DF040
:103A4000E56B90005512444AE0C3951690079EF02E
:103A5000E56B90005812444AE0C3951690079FF01A
:103A6000E56B90005912444AE0C395169007A0F008
:103A7000E56B90005A12444AE0C395169007A1F0F6
:103A8000E56B90005B12444AE0C395169007A2F0E4
:103A9000122BAF7599F9751864751700122B6B808E
:0F3AA000FE7599FF751864751700122B6B80FE69
:093EA1000238C202392002396B1B
:103AAF0022E513903EAAF8282873023BF090078670
:103ABF00E0FEA3E0FF90001212001EE0F5999007C0
:103ACF008612000E900786E0FEA3E0FF74116F4E82
:103ADF007003751300023BF0856299023BF090076B
:103AEF0086E0FEA3E0FF90004E12001EE0F599EF76
:103AFF00B40107EEB4070375130090078612000E8A
:073B0F00023BF0900787E084
:0F3EAA00023AB9023ABC023AE7023AED023B1281
:103B1600903ECBF8282873852499023BE5852A999F
:103B2600023BE5854499023BE5854799023BE585DD
:103B36005199023BE5856099023BE5855699023B22
:103B4600E5855899023BE5756F00900069E07006BF
:103B5600900068E060028016A2A44006E56F440467
:103B6600F56FA2A54006E56F4402F56F801A900036
:103B76004AE0B40106E56F4410F56F900049E0B4E1
:103B86000106E56F4420F56FA207B34006E56F44D2
:103B960001F56FA20CB34006E56F4408F56F856F1B
:103BA60099803CA213B340077599FAC2138017A2F5
:103BB6000FB3400575990F800B900023E0F599909F
:103BC6000023E4F0C20F80178542998012854B9935
:0F3BD600800D85469980087599FC800375130052
:103ECB00023B1D023B23023B29023B2F023B3502E7
:103EDB003B3B023B41023B47023B4D023BA9023BB2
:0D3EEB00CE023BD3023BD8023BDD023BE29E
:0B3BE50090078612000E8003120048BB
:033EB900023BEDDC
:103BF0002290006BE0B4010385241190006BE0B4C7
:103C00000203852A1190006BE0B4030385441190F0
:103C1000006BE0B4040385471190006BE0B405032A
:103C200085511190006BE0B4060385561190006B2E
:103C3000E0B4070385581190006CE0FE90006DE041
:103C4000C39E5003023CC790006BE0D39404402C09
:103C500090006CE0D39511500990006DE0C3951170
:103C600050028002D20090006CE0D3951150099070
:103C7000006DE0C395115002C200804990006BE0D6
:103C8000B4041890006DE0C395115002D20090006A
:103C90006CE0D395114002C200802A90006CE0C312
:103CA0009511500990006DE0D3951150028002D219
:103CB0000090006CE0D39511500990006DE0C39521
:103CC000115002C200807E90006BE0D39404402C1F
:103CD00090006CE0C39511400990006DE0D3951100
:103CE00040028002C20090006CE0C3951140099030
:103CF000006DE0D395114002D200804990006BE046
:103D0000B4041890006CE0C395115002C2009000FA
:103D10006DE0D395114002D200802A90006CE0C380
:103D20009511400990006DE0D395114002D20090AA
:103D3000006CE0D39511400990006DE0C3951140EF
:103D4000028002C2002290006EE0B40103852411BB
:103D500090006EE0B40203852A1190006EE0B40377
:103D60000385441190006EE0B40403854711900070
:103D70006EE0B4050385511190006EE0B406038532
:103D8000561190006EE0B4070385581190006FE063
:103D9000FE900070E0C39E5003023E1C90006EE057
:103DA000D39404402C90006FE0D3951150099000FB
:103DB00070E0C3951150028002D20290006FE0D3F0
:103DC00095115009900070E0C395115002C2028015
:103DD0004990006EE0B40418900070E0C395115053
:103DE00002D20290006FE0D395114002C202802AF5
:103DF00090006FE0C395115009900070E0D39511C9
:103E000050028002D20290006FE0D39511500990C9
:103E10000070E0C395115002C202807E90006EE0F7
:103E2000D39404402C90006FE0C39511400990009A
:103E300070E0D3951140028002C20290006FE0C38F
:103E400095114009900070E0D395114002D2028094
:103E50004990006EE0B4041890006FE0C3951150D3
:103E600002C202900070E0D395114002D202802A73
:103E700090006FE0C395114009900070E0D3951158
:103E80004002D20290006FE0D3951140099000707B
:0B3E9000E0C3951140028002C2022234
:09444A002582F58250020583224F
:10002E00EF2F500205832582F582E5833E2EF58360
:01003E00229F
:08000300C3EF9DFFEE9CFE22FD
:08003F000806B60002180622B3
:0D000E00A3E004F07006124440E004F0226C
:08445C000816B6FF0218162233
:0E442400048007C3CE13CECF13CFD5E0F6220F
:10423C00BC000FBE0008ED8FF084FFADF022E4FE51
:10424C00FF22BE000DEF60FE54F0606F20E703020A
:10425C0042F2EAC0E0EBC0E078017A0075F001EEC2
:10426C0020E710EF25E0FFEE33FE0AC5F023C5F082
:10427C0030E7F0EA5407F9096A7A007B006001081C
:10428C00C3EC9E40167004ED9F4010ED9FFDEC9E1C
:10429C00FCE5F0CA4ACA03F5F08005E5F003F5F039
:1042AC00C3EE13FEEF13FFD9D77908CACBCAD8D007
:1042BC00EAFEEBFFD0E0FBD0E0FA22EC8FF084FCBE
:1042CC00ED54F045F0C48FF084FEEDC454F045F08D
:1042DC00C48FF084FDEEC4FE54F02DFFEE540F3C61
:1042EC00FEADF07C0022790078008FF0EC7E082087
:1042FC00E70DC3CD33CD33C933C9C833C8DEF08421
:10430C0049F9E5F08FF0BE00E6FD7C00E9FFE8FE20
:01431C00227E
:0E443200F88FF0A4FFE5F0CE88F0A42EFE2255
:10440400600D782B02440E007830D8FED5E0F822F7
:10441400EEC0E07E0012423CEFFDEEFCD0E0FE2256
:03000B000243B3FA
:03001B000243CECF
:03002B000243E9A4
:0300000002445364
:0944530075817375D00002082B7D
:0B001E00E5822FF582E5833EF583228A
:0A4440000582D58202158315822241
:1043B300C0E0C0F0C083C082C0D075D00012082016
:1043C300D0D0D082D083D0F0D0E032C0E0C0F0C0F3
:1043D30083C082C0D075D000120823D0D0D082D041
:1043E30083D0F0D0E032C0E0C0F0C083C082C0D040
:1043F30075D000120826D0D0D082D083D0F0D0E080
:014403003286
:00000001FF
